:020000004A288C
:08000800182895201F21D020CB
:10001000EA20352845284528B620132145284528BB
:10002000E22015214528000045284528792045284B
:1000300064009000030E83128F00FC3081000B11CE
:100040008C0B232828280F0E8300900E100E090019
:100050000A308C008D0A0E1C32280F0E8300900E81
:10006000100E09000E148B1705280D1C0A288D1C74
:100070000B280D1D0C288D1D0F280D1E10288D1E00
:1000800013280D1F15288D1F16288B138B1B452831
:100090000E10090019308820831600308500831265
:1000A0000230850083160130860083128601831694
:1000B0005730810083126620FC3081000A308C00AA
:1000C0008B1601308D008E018B176528023085005C
:1000D00000308600950191019201930194019901EC
:1000E0009A019B010230A0000130A400A101A201ED
:1000F0000800950A1508173C031D08008B138B1B7D
:100100007E28023085003230882012308500872812
:1001100096000D309700003098006400980B8E28F0
:10012000970B8B28960B892808001118AA28061807
:100130009B2894010800940A1408023C031D08003F
:1001400011149401920A93019501241C08000430B3
:10015000A0000800061CAE2894010800940A1408A8
:10016000053C031D08001110940108001118BA285D
:10017000930A0800930108008518C0288514080018
:10018000851008001118C6289A010800121CCC28F6
:100190001914FF309A0008001910FF309A00080067
:1001A0009A08031DD6280511851108009A0319180D
:1001B000DC280515851108000511851508009E012C
:1001C0009F0108009F0A1F08B83C031D08009E0AF3
:1001D0009F0108002018F428A018FC2820190429E1
:1001E000A0190C29851408000D087E39031DFA2872
:1001F00085100800851408000D080E39031D02291A
:1002000085100800851408000D080339031D080037
:1002100085100830A00008000D080339031D0800F0
:100220008514A0010800A1030800A2080319080012
:10023000861E1D298612A2030800861608001B08C8
:10024000003C031980291B08013C031988291B085D
:10025000023C03198C291B08033C031996291B082F
:10026000043C03199C291B08053C0319A7291B08FA
:10027000063C0319AD291B08073C0319B8291B08C4
:10028000083C0319BE291B08093C0319C8291B088F
:100290000A3C0319CC291B080B3C0319D3291B0862
:1002A0000C3C0319DB291B080D3C0319E3291B082F
:1002B0000E3C0319EB291B080F3C0319F3291B08FB
:1002C000103C0319FA291B08113C0319FF291B08CC
:1002D000123C0319032A1B08133C03190C2A1B08A0
:1002E000143C0319102A1B08153C0319172A1B0874
:1002F000163C03191F2A1B08173C0319272A7E28BE
:100300000230A0001308023C031D08009B0A0800ED
:10031000111C08009B0A08001308143C031D9429B3
:100320000230A0009B0A0800C2200800111C08002F
:100330009B0A0130920008001308143C031DA629F3
:1003400012089C000230A0009B0A08000800111C43
:1003500008009B0A0130920008001308143C031D9A
:10036000B7291208A3000230A0009B0A0800080069
:10037000111C08009B0A0130920008001308143C6D
:10038000031DC72912089D009B0AA401080008004C
:100390000430A2009B0A0800A208031D08000630D2
:1003A000A1009B0A0800A108031D080006160630DC
:1003B000A1009B0A0800A108031D080006121430C2
:1003C000A1009B0A0800A108031D080006160630BC
:1003D000A1009B0A0800A108031D080006120630B0
:1003E000A1009B0A0800A108031D08000130A2001B
:1003F0009B0A0800A208031D08009B0A0800DF20D2
:100400009B0A201408001D081E020319092A9501E1
:1004100008009B0AA00108000430A2009B0A080003
:10042000A208031D08009B0A0630A1000800A108CD
:10043000031D080006160630A1009B0A0800A1084B
:10044000031D080006129630A1009B0A0800A108AF
:10045000031D0800990135229A0095019C0B322A50
:100460009B0A080013309B0008002308013C031975
:1004700005342308023C03190A342308033C0319FA
:1004800014342308043C031923342308053C0319BE
:1004900037342308063C031946342308073C031964
:0404A0006434873405
:00000001FF
